:03000000020030CB
:03000B0002018867
:1000300075816075A800758C00758A00791E7A003C
:100040007B007C007E00C2D5C2B7C2B5C2B07F3B88
:100050001201AB7F0C1201AB7F011201ABD2B012C7
:1000600001BB7F051201C57F551201AB7F761201DE
:10007000AB7F6F1201AB7F6C1201AB7F6E1201ABD5
:100080007F651201AB7F741201AB7F651201AB7FFC
:10009000451201C57F741201AB7F6C1201AB7F6109
:1000A0001201AB7F631201AB7F691201AB7F741247
:1000B00001AB7F6B1201AB7F611201AB30B4FD303D
:1000C000B3FA7550FF7551FFD551FDD550F71201A8
:1000D000BB7F061201C57F531201AB7F541201ABE7
:1000E0007F411201AB7F521201AB7F541201AB2052
:1000F000B4FD7550FF7551FFD551FDD550F775A86A
:1001000082758902758810D2B730B402C2B7C2D5E1
:100110008A528B538C548E5520D5F330B203120182
:10012000DC30B40312015830B30312016402010938
:10013000E555FF1201707F3A1201ABE554FF120141
:10014000707F3A1201ABE553FF1201707F3A120142
:10015000ABE552FF120170221201A67F031201C506
:10016000120130221201A67F431201C51201302272
:100170001201822430FF1201ABE5F02430FF12019E
:10018000AB22EF75F00A8422C0D0D917791E0AD2AB
:10019000D5BA640F7A000BBB3C097B000CBC3C0356
:1001A0007C000ED0D03278FFD8FE221201A68F90AC
:1001B000D2B11201A6C2B11201A622C2B07F0112B1
:1001C00001ABD2B022C2B01201A6EF4480FF8F90E3
:1001D0001201AB1201A6D2B01201A622AF53E5550F
:1001E0007004E554601CE5540475F00584E5F07076
:1001F0000ABF3202D2B5BF3B02D2B7BF0004C2B5BC
:05020000C2B70000225E
:00000001FF
